:100000000C945D000C9485000C9485000C94850084
:100010000C9485000C9485000C9485000C9485004C
:100020000C9485000C9485000C9485000C941304AA
:100030000C9485000C9485000C9485000C9485002C
:100040000C94C9030C9485000C9497030C947103D1
:100050000C9485000C9485000C9485000C9485000C
:100060000C9485000C94850000000008000201003B
:100070000003040700000000000000000000000072
:10008000250028002B0000000000240027002A0083
:10009000040404040404040402020202020203032E
:1000A0000303030301020408102040800102040836
:1000B0001020010204081020EA0411241FBECFEF13
:1000C000D8E0DEBFCDBF11E0A0E0B1E0EEE6FEE09B
:1000D00002C005900D92A433B107D9F722E0A4E342
:1000E000B1E001C01D92AD30B207E1F710E0CDE5FF
:1000F000D0E004C02197FE010E942F07CC35D10724
:10010000C9F70E9422050C9435070C94000090E07A
:10011000FC01EC55FF4F249180579F4FFC018491C7
:10012000882399F090E0880F991FFC01EA57FF4F50
:10013000A591B491FC01E458FF4F859194918FB73C
:10014000F894EC91E22BEC938FBF08951F93CF931B
:10015000DF93EC01162F88818C3008F04DC0862F7C
:100160000E9487008881282F30E0F901EE0FFF1FE1
:10017000E20FF31FED5BFE4F1F736081607C612B0C
:10018000608319821A822CE0622F0E942307829FCB
:10019000B001112430E020E0AB01420F531FFA01FF
:1001A000EE0FFF1FE40FF51FED5BFE4F908196FDF4
:1001B00016C02F5F3F4F2C30310571F781110FC0F2
:1001C0001092800082E0809381001092850010924E
:1001D0008400B19A80916F00826080936F00E88103
:1001E0008E2F90E0FC01EE0FFF1FE80FF91FED5B73
:1001F000FE4F8081806480838881DF91CF911F9141
:100200000895AF92BF92CF92DF92EF92FF920F9339
:100210001F93CF93DF936C017B018B01040F151F9C
:10022000EB015E01AE18BF08C017D10759F0699104
:10023000D601ED91FC910190F081E02DC601099568
:10024000892B79F7C501DF91CF911F910F91FF9015
:10025000EF90DF90CF90BF90AF900895FC01538D49
:10026000448D252F30E0842F90E0821B930B541790
:1002700010F0CF96089501970895FC01918D828D1D
:10028000981761F0A28DAE0FBF2FB11D5D968C91B6
:10029000928D9F5F9F73928F90E008958FEF9FEFF5
:1002A0000895FC01918D828D981731F0828DE80FB1
:1002B000F11D858D90E008958FEF9FEF08952FB782
:1002C000F89480913F0190914001A0914101B0913B
:1002D00042012FBF80936F0190937001A093710131
:1002E000B093720187E691E00E94510197FF26C00A
:1002F0002FB7F89480913F0190914001A091410166
:10030000B09142012FBF40916F01509170016091F7
:10031000710170917201841B950BA60BB70B409174
:100320006B0150916C0160916D0170916E018417A9
:100330009507A607B707B0F28FEF9FEF0895FC016E
:10034000918D228D892F90E0805C9F4F821B9109B7
:100350008F739927089587E691E00E949F0121E01D
:10036000892B09F420E0822F089580E090E0892B0A
:1003700029F00E94AB0181110C9400000895FC014A
:10038000A48DA80FB92FB11DA35ABF4F2C91848DF6
:1003900090E001968F739927848FA689B7892C9353
:1003A000A089B1898C91837080648C93938D848DA6
:1003B000981306C00288F389E02D80818F7D8083A9
:1003C0000895EF92FF920F931F93CF93DF93EC0169
:1003D00081E0888F9B8D8C8D98131AC0E889F989EC
:1003E000808185FF15C09FB7F894EE89FF896083EF
:1003F000E889F98980818370806480839FBF81E070
:1004000090E0DF91CF911F910F91FF90EF900895B1
:10041000F62E0B8D10E00F5F1F4F0F731127E02E8C
:100420008C8D8E110CC00FB607FCFACFE889F989C4
:10043000808185FFF5CFCE010E94BF01F1CFEB8D0A
:10044000EC0FFD2FF11DE35AFF4FF0829FB7F89498
:100450000B8FEA89FB8980818062CFCFCF93DF93B6
:10046000EC01888D8823B9F0AA89BB89E889F989CC
:100470008C9185FD03C0808186FD0DC00FB607FC01
:10048000F7CF8C9185FFF2CF808185FFEDCFCE0134
:100490000E94BF01E9CFDF91CF91089590E0FC0168
:1004A000E859FF4F2491FC01EC55FF4F3491FC01BA
:1004B000E057FF4FE491EE23C9F0222339F02330B7
:1004C00001F1A8F4213019F1223029F1F0E0EE0F0A
:1004D000FF1FE458FF4FA591B4918FB7F894EC91AA
:1004E000611126C030953E233C938FBF089527307D
:1004F000A9F02830C9F0243049F7809180008F7D21
:1005000003C0809180008F7780938000DFCF84B517
:100510008F7784BDDBCF84B58F7DFBCF8091B0001A
:100520008F778093B000D2CF8091B0008F7DF9CFCC
:100530003E2BDACF3FB7F894809137019091380184
:10054000A0913901B0913A0126B5A89B05C02F3F73
:1005500019F00196A11DB11D3FBFBA2FA92F982FE9
:100560008827BC01CD01620F711D811D911D42E0E4
:10057000660F771F881F991F4A95D1F708958F92AC
:100580009F92AF92BF92CF92DF92EF92FF920E9422
:100590009A024B015C0180EBC82E84E0D82EE12C3E
:1005A000F12C0E949A02681979098A099B09683E10
:1005B000734081059105A8F321E0C21AD108E10832
:1005C000F10888EE880E83E0981EA11CB11CC114AE
:1005D000D104E104F10429F7FF90EF90DF90CF9070
:1005E000BF90AF909F908F900895CF92DF92EF923F
:1005F000FF92CF93DF93EC01603282E07807CCF575
:10060000653B710514F064EB70E0898128E830E007
:10061000281B310987FD3395220F331F220F331F0B
:100620006901330FEE08FF088A8128E532E0281BB4
:10063000310987FD3395220F331F220F331F032EFD
:10064000000C440B550B2C193D094E095F09DB01C9
:1006500077FF02C0B0E0A0E00E94EA0624EB30E0A1
:1006600040E050E00E94C006C20ED31EE41EF51EFC
:10067000B601E881EC3070F5298188E890E0821BB2
:10068000910927FD9395880F991F880F991F681767
:1006900079077CF02A8188E592E0821B910927FD89
:1006A0009395880F991F880F991F681779070CF485
:1006B000CB010297880F991F4FB7F8942E2F30E087
:1006C000F901EE0FFF1FE20FF31FED5BFE4F928368
:1006D00081834FBFDF91CF91FF90EF90DF90CF905C
:1006E00008951F920F920FB60F9211242F933F93EC
:1006F0004F935F936F937F938F939F93AF93BF932A
:10070000EF93FF9387E691E00E94BF01FF91EF9185
:10071000BF91AF919F918F917F916F915F914F9119
:100720003F912F910F900FBE0F901F9018951F9221
:100730000F920FB60F9211242F938F939F93EF93E5
:10074000FF93E0917701F09178018081E0917D0144
:10075000F0917E0182FD1BC09081809180018F5FAE
:100760008F7320918101821741F0E0918001F0E0C8
:10077000E959FE4F958F80938001FF91EF919F91F2
:100780008F912F910F900FBE0F901F901895808121
:10079000F4CF1F920F920FB60F9211242F933F9315
:1007A0008F939F93AF93BF9380913F0190914001AE
:1007B000A0914101B09142013091360123E0230F15
:1007C0002D3758F50196A11DB11D20933601809358
:1007D0003F0190934001A0934101B0934201809169
:1007E000370190913801A0913901B0913A010196F9
:1007F000A11DB11D8093370190933801A093390159
:10080000B0933A01BF91AF919F918F913F912F91FA
:100810000F900FBE0F901F90189526E8230F029699
:10082000A11DB11DD2CF1F920F920FB60F921124AE
:100830002F933F934F935F936F937F938F939F93E8
:10084000AF93BF93CF93DF93EF93FF9380913401E6
:10085000C0913501D0E087FF24C01092850010922E
:100860008400809134018F5F809334018091340142
:10087000082E000C990B8C179D0724F480913401ED
:100880008C30C4F18091840090918500049680346E
:100890009C4908F47AC08091840090918500049668
:1008A00076C080913401082E000C990B8C179D079F
:1008B000C4F6E09134018E2FEE0F990BFC01EE0F80
:1008C000FF1FE80FF91FED5BFE4F808186FFC9CF48
:1008D000E09134018E2FEE0F990BFC01EE0FFF1FFC
:1008E000E80FF91FED5BFE4F808160E08F730E947F
:1008F0004E02B7CF2091840030918500E091340101
:100900008E2FEE0F990BFC01EE0FFF1FE80FF91F62
:10091000ED5BFE4F81819281820F931F909389003E
:1009200080938800E09134018E2FEE0F990BFC012B
:10093000EE0FFF1FE80FF91FED5BFE4F808186FF72
:1009400011C0E09134018E2FEE0F990BFC01EE0FD8
:10095000FF1FE80FF91FED5BFE4F808161E08F7391
:100960000E944E02FF91EF91DF91CF91BF91AF9125
:100970009F918F917F916F915F914F913F912F91B7
:100980000F900FBE0F901F90189580E49CE99093F4
:100990008900809388008FEF80933401E3CFFC01BE
:1009A000909135019C3098F481E0890F8093350156
:1009B0009083892F90E0FC01EE0FFF1FE80FF91FD5
:1009C000ED5BFE4F88EB9BE09283818308958FEF70
:1009D00080830895E7E6F1E01382128288EE93E0C7
:1009E000A0E0B0E084839583A683B78384E091E0A0
:1009F0009183808385EC90E09587848784EC90E0F8
:100A00009787868780EC90E0918B808B81EC90E0DB
:100A1000938B828B82EC90E0958B848B86EC90E0BC
:100A2000978B868B118E128E138E148E8AE092E035
:100A30000E94CF0487E092E00E94CF0484E092E01D
:100A40000C94CF04789484B5826084BD84B58160B1
:100A500084BD85B5826085BD85B5816085BD809189
:100A60006E00816080936E00109281008091810001
:100A700082608093810080918100816080938100F9
:100A8000809180008160809380008091B1008460BB
:100A90008093B1008091B00081608093B00080911C
:100AA0007A00846080937A0080917A0082608093DB
:100AB0007A0080917A00816080937A0080917A0038
:100AC000806880937A001092C100E0917701F091E4
:100AD000780182E08083E0917301F09174011082CB
:100AE000E0917501F091760187E6808310927F0195
:100AF000E0917B01F0917C0186E08083E0917901B7
:100B0000F0917A01808180618083E0917901F09198
:100B10007A01808188608083E0917901F0917A0187
:100B2000808180688083E0917901F0917A018081F1
:100B30008F7D8083C0E0D0E087E691E00E949F0136
:100B4000892B09F44DC00E945F01FC0197FDFBC099
:100B50008D32910521F0C0970A9708F0EDC0C12CA5
:100B6000D12C760110E0E130F105D9F0ED32F1053C
:100B700009F4E7C0CF01C0970A9798F4AAE0B0E063
:100B8000A70196010E94DF066F01FF0FEE08FF0824
:100B9000C60ED71EE81EF91E80E3C81AD108E10868
:100BA000F10887E691E00E943D010E945F01FC018F
:100BB000C0970A97C0F2E130F105A9F2112341F084
:100BC000F094E094D094C094C11CD11CE11CF11CA1
:100BD000C0923B01D0923C01E0923D01F0923E0177
:100BE000C0903B01D0903C01E0903D01F0903E016F
:100BF000D701C6010197A109B109853B9105A1055E
:100C0000B10520F569E070E08AE092E00E94A6005C
:100C1000B601615071098AE092E00E94F5020E94DB
:100C2000BF02E0910A028E2F90E0FC01EE0FFF1F41
:100C3000E80FF91FED5BFE4F80818F7B808389E099
:100C40000E94870060E089E00E944E02D701C60141
:100C5000895E9340A109B109853B9105A105B105C4
:100C600020F56AE070E087E092E00E94A600B601FD
:100C7000695E734087E092E00E94F5020E94BF0225
:100C8000E09107028E2F90E0FC01EE0FFF1FE80FAE
:100C9000F91FED5BFE4F80818F7B80838AE00E948D
:100CA000870060E08AE00E944E02D701C601815DA4
:100CB0009740A109B109853B9105A105B10508F04F
:100CC00046C06BE070E084E092E00E94A600B601AE
:100CD000615D774084E092E00E94F5020E94BF02CD
:100CE000E09104028E2F90E0FC01EE0FFF1FE80F51
:100CF000F91FED5BFE4F80818F7B80838BE00E942C
:100D0000870060E08BE00E944E0287E691E00E943F
:100D10002E0210923B0110923C0110923D01109264
:100D20003E01209709F408CF0E94AB01882309F403
:100D300003CF0E94000000CF87E691E00E943D01B2
:100D400002CF11E02ECFC12CD12C760141CF81E60C
:100D5000C81683EED80686E1E806F104B1F64EE146
:100D600050E062E171E087E691E00E94010142E01B
:100D700050E061E371E087E691E00E940101C5CF98
:100D8000052E97FB1EF400940E94D70657FD07D04E
:100D90000E94F20607FC03D04EF40C94D70650953F
:100DA0004095309521953F4F4F4F5F4F0895909557
:100DB0008095709561957F4F8F4F9F4F08950E944A
:100DC0001407A59F900DB49F900DA49F800D911DB9
:100DD00011240895B7FF0C94DF060E94DF06821BE2
:100DE000930B0895A1E21A2EAA1BBB1BFD010DC097
:100DF000AA1FBB1FEE1FFF1FA217B307E407F507CB
:100E000020F0A21BB30BE40BF50B661F771F881FA6
:100E1000991F1A9469F760957095809590959B013C
:100E2000AC01BD01CF010895A29FB001B39FC001E5
:100E3000A39F700D811D1124911DB29F700D811D06
:100E40001124911D0895991B79E004C0991F9617EC
:100E500008F0961B881F7A95C9F780950895EE0FC4
:0E0E6000FF1F0590F491E02D0994F894FFCF48
:100E6E0000000000E10101012E012E029F013D0153
:100E7E00510157616E64657265724D61737465726E
:100E8E0054696C74657241323032323037333141CD
:040E9E00000D0A0039
:00000001FF
